:1000000028C041C013C23FC084C13DC03CC03BC0FA
:100010003BC121C138C007C336C035C03FC233C061
:1000200032C031C030C05EC048C0D2C046C067C018
:1000300077C088C098C0ACC040C0B1C03EC0DCC072
:100040003CC0ABC398C39CC39EC3A2C3A6C393C307
:10005000A7C311241FBECFE5D4E0DEBFCDBF11E0A2
:10006000A0E6B0E0E6EBFCE002C005900D92AC35F6
:10007000B107D9F711E0ACE5B1E001C01D92AE3691
:10008000B107E1F701C0BCCFCFE5D4E0DEBFCDBF03
:1000900011E0109362018AD310926B01BBD39BD302
:1000A000A3D3ADD38FB780688FBF10936C0182E06C
:1000B00080935F0180E28093600180916C018823CE
:1000C00021F08093690110926C0180916901992758
:1000D000AA27BB27FC013197EE30F10570F7ED5EE2
:1000E000FF4F099482E08093690192D084B38360CA
:1000F00084BB85B38C7F85BB9798A0D0DECF88D09A
:100100008ED089B7856089BF86B186E886B984B309
:10011000836084BB85B38C7F85BB979886E075C070
:1001200087B18377836687B9369A3699FECF85B1D2
:100130008093680187B18277826687B9369A36994B
:10014000FECF22C065D06BD089B7856089BF86B1EC
:1001500086E886B984B38C7F84BB85B38C7F85BBEE
:10016000979A88E052C087B18177816687B9369ABD
:100170003699FECF85B18093680187B1807780661C
:1001800087B9369A3699FECF85B180935C0195CFB9
:100190003FD045D089B7856489BF8AE036C038D062
:1001A0003ED01092680110925C0184B3836084BBDE
:1001B00085B38C7F85BB979889E080936A0126D3AD
:1001C00012BE1DBC1CBC14BC8CE08093690110C025
:1001D0001FD082B3806382BB88B3806388BB1FD08B
:1001E00030D3579A84E0809369018FE480936A0149
:1001F00089B7856489BF61CF0BD082B3806382BB2E
:1002000088B3806388BBA4D28EE08093690155CF08
:1002100089B78A7B89BF579833985498089510926C
:1002200064011092670110926A0182B3806382BBFD
:1002300088B3806388BBC19AC29A0895F0DF109298
:100240006D0183E680936A0188B7856488BF89B7AA
:10025000856489BF08951F920F920FB60F921124E3
:100260008F938091680182BF959B04C082B38F7D7C
:10027000806103C082B38F7E806282BB8F910F90BA
:100280000FBE0F901F9018951F920F920FB60F92EE
:1002900011248F939F9380915C0199279DBD8CBD04
:1002A000C59B04C088B38F7D806103C088B38F7EF7
:1002B000806288BB9F918F910F900FBE0F901F900F
:1002C000189589B78E7F89BF82B3806382BB0895FA
:1002D00080916301E0E6F0E0E80FF11D80818093FA
:1002E000680189B7816089BF089589B78B7F89BF0D
:1002F00088B3806388BB089580916601E0E6F0E0F2
:10030000E80FF11D808180935C0189B7846089BF0B
:1003100008951F920F920FB60F9211242F933F93BF
:100320004F935F936F937F938F939F93AF93BF93FD
:10033000EF93FF9320916A012F5F20936A018091D0
:10034000690199278430910509F45BC085309105D6
:100350001CF4029739F059C08A30910561F10C976D
:10036000C1F153C0243609F050C010926A01F6D191
:1003700090916D01A92FBB27FD01E157FF4FE0814F
:10038000E0936301AD50BF4F8C91809366019F5FF6
:1003900090936D01EF3F21F48DE080936C0135C0A7
:1003A000E33611F48EDF01C093DF8091660183365E
:1003B00059F1A2DF2AC0243141F510926A01CED151
:1003C000A7D2DC01CB0180936801A2D2DC01CB0172
:1003D00015C02A30D1F410926A01809168018F5FB4
:1003E00080936801803F10F01092680180915C0159
:1003F000815080935C01803F40F080EF80935C01EE
:1004000004C0203511F45DDF70DFFF91EF91BF91E3
:10041000AF919F918F917F916F915F914F913F919C
:100420002F910F900FBE0F901F9018951F920F9253
:100430000FB60F9211242F933F934F935F936F93B7
:100440007F938F939F93AF93BF93EF93FF938BB75C
:100450008F778BBFDDDE82B3806382BB88B380631E
:1004600088BB8B9A939A86E090E04ED187B18475D1
:10047000846487B9349A339A369AFF91EF91BF9189
:10048000AF919F918F917F916F915F914F913F912C
:100490002F910F900FBE0F901F9018951F920F92E3
:1004A0000FB60F921124EF92FF920F931F932F9389
:1004B0003F934F935F936F937F938F939F93AF93EC
:1004C000BF93CF93EF93FF93339824B185B19927CE
:1004D000182F0027020F111DC801AA2797FDA0950C
:1004E000BA2FBC01CD01D5D217FF05C020E030E006
:1004F00040E857E421D29B01AC0160E070E080E865
:1005000094E464D2DC01CB0120E030E040E85FE31A
:10051000BC01CD0110D2DC01CB0120E030E04CE782
:1005200052E4BC01CD0101D3DC01CB0120E030E07D
:1005300040E05FE3BC01CD01FFD1DC01CB01BC0198
:10054000CD018AD27B018C01C62F85B7837F85BF01
:100550008B98939882E090E0D7D085B78B7F8860A6
:1005600085BF8BB780688BBF8091600190916901D6
:10057000E81651F49E3061F48E2D992786729070A2
:10058000892B71F0D4D00CC0E09260019E3011F044
:100590008DE031C083B7816083BF8EB581608EBD31
:1005A000C09360018C2F992784309105E9F0853044
:1005B000910534F481309105E1F00297B9F01DC046
:1005C0008031910551F0813191051CF4089741F07B
:1005D00014C0809791F481E00EC0969A85E00BC01C
:1005E000C09A929A87E007C089E005C0929A8BE092
:1005F00002C0C09A83E080936C01FF91EF91CF918C
:10060000BF91AF919F918F917F916F915F914F912A
:100610003F912F911F910F91FF90EF900F900FBE80
:100620000F901F9018951F920F920FB60F921124E2
:100630002F933F934F935F936F937F938F939F93EA
:10064000AF93BF93EF93FF9388B331E0832788BBC9
:1006500082B394E0892782BB5C9945C02CB1822F7C
:1006600099278133910579F08137910589F403B693
:1006700000FE39C090E080916201882309F4932F35
:100680009093620130C053D02EC0E0936B012BC019
:1006900080E0A82FBB27FD01E658FF4FE081EE2345
:1006A000A1F3E217F1F4A05ABF4F8C918093680137
:1006B0008F5F80935C0110926A0189B7816089BF66
:1006C00081E090E021D003B600FE04C08091620179
:1006D000882319F089B7846089BF89B7806489BF8E
:1006E00002C08F5FD6CFFF91EF91BF91AF919F91E5
:1006F0008F917F916F915F914F913F912F910F90CB
:100700000FBE0F901F90189540E050E04817590712
:1007100068F420E030E0275E3F4F60E72E34360774
:10072000D0F34F5F5F4F4817590798F3089503B60A
:1007300000FE06C083B78E7F83BF8EB58E7F05C057
:1007400083B7816083BF8EB581608EBD08950895A3
:10075000A998A8989298C09896980895D9D0DC0145
:10076000CB0187709070A070B070FC010897E0F426
:10077000EF5DFF4F099485B391E0892785BB08950C
:1007800082B394E007C088B391E0892788BB0895BD
:1007900082B390E4892782BB089585B392E0EDCFC0
:1007A00082B390E4892782BB0895089587B38F634D
:1007B00087BB88B3807F806388BB84B3837C83607E
:1007C00084BB85B3807C85BB81B386EF81BB82B35C
:1007D00082E382BB089583B78B7F836083BF89B731
:1007E0008E7F89BF12BE08958FB581E08FBD8EB513
:1007F0008B728B608EBD89B7837C89BF089585B568
:1008000085E085BD89B78F7389BF089580B7836000
:1008100080BF089585B715BE8B989398A498AC981F
:1008200082E090E071DF8AB780688ABF8BB780680A
:100830008BBF86B186E986B987B18475846487B930
:1008400008958BB1807E80648BB98AB1827180619A
:100850008AB986E880BD80B5807780BD8FEC89B984
:100860000895A0E0B0E0E6E3F4E0F6C1EC01E88032
:10087000F9800A811B81C801B7012DE133EF41E006
:1008800050E0C0D159016A01C801B7012DE133EF31
:1008900041E050E0B7D1DC01CB01BC01CD0127EA3A
:1008A00031E440E050E08FD17B018C01C601B501FD
:1008B00024E13BE040E050E086D1DC01CB01E81AC6
:1008C000F90A0A0B1B0B1E141F041006110644F034
:1008D0008FEF9FEFAFEFBFE7E80EF91E0A1F1B1F58
:1008E000E882F9820A831B838FEF9FEFAFEFBFE7A8
:1008F000E822F9220A231B23C801B701EAE0CDB799
:10090000DEB7C6C1AEDFDC01CB01BC01CD0108956D
:1009100087E591E0A6DFDC01CB01BC01CD010895A4
:10092000DC01CB018093570190935801A0935901AA
:10093000B0935A0108955058192ED5D001D0B8C09F
:10094000BA176207730784079507B1F188F40EF4AC
:1009500010940B2EBA2FA02D062E622F202D072EBD
:10096000732F302D082E842F402D092E952F502DBA
:10097000FF275523B9F0591B49F0573E98F046958B
:1009800037952795A795F0405395C9F776F0BA0F9C
:10099000621F731F841F30F4879577956795B7950D
:1009A000F040939517FA0F2E0895BF1BBB27BA0B83
:1009B000620B730B840BF6CFDEF6B1C0592F482FB4
:1009C000372F262F9FE380E8772766278CD001D02A
:1009D0006FC0552359F0992369F09F575F57951BB6
:1009E00033F442F4903811F4915805C079C091580D
:1009F0009F3F09F494C0BB27112462177307840733
:100A000030F4660F771F881FBB1F915098F311D0E9
:100A10000F920FD00F920DD0A0E826173707480786
:100A20001B0609F0A048BA2F602D7F918F910024FA
:100A30000895A0E80024621773078407B10528F021
:100A4000621B730B840BB1090A2A660F771F881F7C
:100A5000BB1FA69581F7089597FB51D09F3738F0BB
:100A6000FEE9F91B982F872F762F6B2F05C054C0F6
:100A70009695879577956795F150D0F73EF49095C8
:100A80008095709561957F4F8F4F9F4F0895E894A3
:100A900003C097FB0EF4F3DFB62F672F782F892F53
:100AA0009EE9002405C09A95BB0F661F771F881F1B
:100AB00011249923A1F08823B2F79F3F59F0BB0F6F
:100AC00048F421F4002011F460FF04C06F5F7F4FF1
:100AD0008F4F9F4F881F9795879597F908951CC052
:100AE0009FEF80EC0895052E092607FA440F551F45
:100AF0005F3F79F0AA27A51708F051E04795880FC6
:100B0000991F9F3F31F0BB27B91708F091E08795F7
:100B100008959F919F91E4CF66277727882799278B
:100B20000895592F482F372F262FDDDF01D0C0CF52
:100B3000992339F0552329F09F575F57950F13F4E8
:100B4000CAF1EDCF91589F3FE1F3A62F0024112465
:100B5000BB2766275527F8E0A69520F4020E131E42
:100B6000B41F651F220F331F441F551FFA95A1F7AD
:100B7000F8E0E72F7727F8E0E69520F4130EB41F8E
:100B8000651F7A1F330F441F551FAA1FFA95A1F73F
:100B9000F82F8827F69520F4B40F651F7A1F8E1F53
:100BA000440F551FAA1FEE1FFF23A1F788231AF435
:100BB000939539F495CF000C111CBB1F661F771F4E
:100BC000881F01280895629FD001739FF001829FC2
:100BD000E00DF11D649FE00DF11D929FF00D839FCC
:100BE000F00D749FF00D659FF00D9927729FB00D69
:100BF000E11DF91F639FB00DE11DF91FBD01CF017C
:100C000011240895A1E21A2EAA1BBB1BFD010DC0E1
:100C1000AA1FBB1FEE1FFF1FA217B307E407F507AC
:100C200020F0A21BB30BE40BF50B661F771F881F88
:100C3000991F1A9469F760957095809590959B011E
:100C4000AC01BD01CF0108952F923F924F925F9268
:100C50006F927F928F929F92AF92BF92CF92DF92CC
:100C6000EF92FF920F931F93CF93DF93CDB7DEB731
:100C7000CA1BDB0B0FB6F894DEBF0FBECDBF0994C5
:100C80002A88398848885F846E847D848C849B841C
:100C9000AA84B984C884DF80EE80FD800C811B812A
:100CA000AA81B981CE0FD11D0FB6F894DEBF0FBE59
:060CB000CDBFED01089527
:100CB60003111E2B37424D576169727A81888F96D0
:100CC6009CA1A6ACB0B5B9BDC1C4617365647266BA
:100CD600677968756A696B6C703B5B275C00000816
:100CE6000A0C0F0D0D110F0F1413140F0C080A0C1C
:100CF6000D0F110F0D0C0A0C0807080A03070A0D41
:100D06000C0A0C080A0C0F0D0D110F0F1413140FFB
:100D16000C080A0C050F0D0C0A08030807080C0F2F
:100D2600140F0C080C0F08080863FF0000000000F1
:100D360000000000000000000000000000000000AD
:100D46000000006363636363636363636363636396
:100D5600636363636363636363636363636363635D
:100D660063636363636303030708080708080A0CE1
:100D76000C0A0C0C080505080A0A070808050A0AE1
:100D8600010000080C0C0F14140A00000063FF0099
:100D9600000000000000000000000000000000004D
:0C0DA60000000000000000010000000040
:00000001FF
